:020000040000FA
:100000000128831600308500E0308600831211102D
:100010000530940003308600E8208601E820940B28
:100020000A28920193010A308F00083090000F08CF
:100030008500861B3320061B5C20861A7520D22083
:10004000900B172812088E209000920A12081A3C72
:10005000031992011308A9208F00930A1308283C62
:100060000319930117280F308500033094000614FC
:100070008610E82006108614E820940B3728061016
:100080008610053085000A309400E820940B45283E
:1000900011185328093085000A309400D220940B9F
:1000A0004E2811145B28063085000A309400D220B7
:1000B000940B5728111008000F308500033094006E
:1000C0008614E8208610E820940B6028053085000F
:1000D0000A309400E820940B6A280B308500053024
:1000E0009400D220940B712808000F308500033053
:1000F00094000614E8200610E820940B79280530B7
:1001000085000A309400E820940B83280E30850087
:1001100005309400D220940B8A2808008207053409
:1001200009340D340D3405340D34053409340534E7
:1001300005340D340934053405340D340D340D34D3
:10014000053405340D3409340D34053409340D34C7
:100150000D3482070B340A340E340A340F340F3452
:1001600006340A3409340A340E340B340F340A349A
:10017000093406340A340F340A340E340A340B348A
:100180000A3409340A340F340A3406340F340A347A
:100190000B340A340E340F340A340E340F340A345C
:1001A000063409340518D9280519DE2806108610EA
:1001B000E3280519E12806148610E32806108614A2
:1001C000E32806108610E82006108610E8200800B4
:1001D00002308C0000308D0000308E0000008E0B4D
:0C01E000EE288D0BEC288C0BEA280800A0
:02400E00FA3F77
:00000001FF
